:080000000C9470000C94000048
:100008000C9400000C9400000C9400000C94000068
:100018000C9400000C947E070C9400000C940000D3
:100028000C9400000C9400000C9400000C94000048
:100038000C9400000C9400000C94FE000C9400003A
:100048000C94FD040C9400000C9435050C940000ED
:100058000C9400000C9400000C9400000C94000018
:100068000C9400000C9400000C9400000C94000008
:100078000C94EC050C9400000C9427070C940000D9
:100088000C940000000102040810204080003F0684
:100098005B4F666D7D077F6F777C585E7971407323
:1000A8001027E80364000A00010000100001100096
:1000B800010025642E2532640000256400253032B5
:1000C800580025313064000001002D4E414E0000DB
:1000D8000100F80AD0000000F894EE27ECBBF1E02C
:1000E800F5BFE5BFE0936C00F8E1F1BDE1BD8DE03F
:1000F800A2E0BB27ED938A95E9F780E090E1A0E0C4
:10010800B1E0ED930197E9F7E8EDF0E0859195917D
:10011800009761F0A591B59105901590BF01F00188
:1001280005900D920197E1F7FB01F0CFEFEFEDBFDE
:10013800E0E1EEBFC0E0D5E00C9491021A930A9377
:10014800AD81A23130F4ED81F0E0EA56FF4F149111
:1001580001C010E0EB81E03009F01058AC81A23109
:1001680030F4EC81F0E0EA56FF4F049101C000E062
:10017800EA81E03009F0005810950095E12FE06F12
:10018800E0936200E12FE695E695E36CE3B9E02F92
:10019800E295EF60E8BBE02FE07FE360E2BB0C9400
:1001A8006903E0B1E07FE295EF700E2EA0E0B09910
:1001B800A1E0EA2FE295E07F0E0EA0E0B199A1E060
:1001C800EA2FE795E0E0E7950E0EA0E0B299A1E0EE
:1001D800EA2FE295E07FEE0F0E0EA0E0B399A1E0C2
:1001E800EA2FE295E07FEE0FEE0FE00DE095E09349
:1001F800740808950A921A92FA926A937A938A93E3
:100208009A93AA93BA93EA93FA93EFB7EA93E2EB35
:10021800E2BF789436D2E0917508EF5FE0937508F5
:10022800A0917508AE3149F4A0917608E3E8EA2771
:10023800E0937608E0E0E0937508E991EFBFF99163
:10024800E991B991A9919991899179916991F990D7
:100258001990099018950E94080CA0915106A7358D
:1002680011F00C94B001A0914A05A13011F00C9442
:10027800AD01A0915206A230A1F1E2E00E94550A18
:10028800A0915206A63021F5E0E0E0937B080E9499
:100298005E0A0E94640A29F4D9011196E2E0EC93FF
:1002A80017C0E23081F4F901A681B781119719F4DA
:1002B8000E946C0A07C0D9011696ED91FD913197FD
:1002C800FE93EE9305C0E33019F4E1E0E0934A05AC
:1002D800A0917B08A43028F00E946C0AE0E0E0932B
:1002E8007B08A0915206A230A1F5E0E0E0937B08DC
:1002F800CDD1E0937E08F0937F08E0915406E33572
:1003080061F4E0915506E43541F4E0915606EF3486
:1003180021F4E0915706E03509F017C0E2E0E093D8
:100328004A050E945E0AEC5FFA4FDF01EC91EF5F2D
:10033800EC930E945E0AEC5FFA4FE081E43610F01D
:100348000E946C0AEFEFE0937708E6E0EA930E94D8
:100358005505E0E0E0935106A0914A05A13039F433
:100368000E94740AE4E6F0E00E947B0A09F40CC0DB
:10037800E0E0E0934A05A0917B08A43028F00E94B1
:100388006C0AE0E0E0937B08A0914A05A23039F4BA
:100398000E94740AEAE0F0E00E947B0A09F403C0B4
:1003A800E0E0E0934A05A0914A05A03031F4E091DD
:1003B8004805A0914905EA1709F46FC00E945E0A32
:1003C8000E94640A89F40E94810AEAE2EA930E9480
:1003D800F607D9011496EC910E948B0AEBE40E946F
:1003E800940A0E949B0A57C0E230E9F50E94810AEC
:1003F800F901A581A13011F4E4E501C0EAE2EA932C
:100408000E94F607F901A281B381E4E6F0E00E94B8
:10041800D20BFA93EA93E2E0F0E0FA93EA930E94AF
:100428000708F901A281B381E4E6F0E00E94CA0B53
:100438001E2F103021F4EAE2EA930E94F6071130E9
:1004480021F4E3E2EA930E94F607123021F4E6E28F
:10045800EA930E94F6070E945008E1E00E94550ABC
:100468000E949B0A18C0E330C1F40E94810AE3E5A8
:10047800EA930E94F607F901A481E4E60E94CF0BF3
:100488000E948B0AE3E50E94940AE0917B08EF5FE3
:10049800E0937B08ECE0E09377080E940F0C249629
:1004A80008951A93A8950E94A408E13041F4E1E068
:1004B800E0937908EBD0E0937C08F0937D0862D153
:1004C8001E2FE0917A08E11731F010937A08E09135
:1004D8007A08E0937808E0917C08F0917D08FA9317
:1004E800EA93EFE0F0E00E947B0A19F0E0E0E09385
:1004F80079080E94A20AE09179080E94A90A0E943C
:10050800A108A9DEE0917608E07829F0E091760864
:10051800EF77E093760819910895E0E0E5BFE0935E
:100528006D00E0936C00EFEFEBBBEABBE8BBE0EFDC
:10053800E7BBE0EDE5BBEFEDE4BBE3EFE2BBE8EFE3
:10054800E1BBEFEFE3B9EEE7E2B9EFEFE09362006A
:10055800EFE0E0936100EFEFE0936500EFE1E093F7
:100568006400E0E0E0BFE7E0E3BFE2EBE2BFE0E029
:10057800E1BFEFBDEEBDEDBDECBDE7BDE6BDEBBD3A
:10058800EABDE9BDE8BDE0937900E0937800E5BDF8
:10059800E4BDE3BDE0938B00EAE0E0938A00E0E08D
:1005A800E0938900E0938800E0938100E093800065
:1005B800E2E1E0938700E4E3E0938600E0E0E09383
:1005C8008500E0938400E0938300E0938200E09349
:1005D8006A00EABFE9BFE1E0E7BFE0E0E0937D0041
:1005E800E0DDE0E0EBB9E8EDEAB9E6E2E09395009A
:1005F800E0E0E0939000EEECE9B9E0E0E0939B00E6
:10060800E8EDE0939A00E6E0E0939D00E0E0E093F7
:100618009800E0917408E87011F0E3E301C0E7E6A0
:10062800E0939900E0E8E8B9E0E0E0BDEEE1E1BD83
:10063800EEE0E1BDE1E0E0937708E09378080E94FE
:10064800A20AE0E00E94A90AE4EFF1E0FA93EA9333
:100658000E94830BEFEFE0937708E09378080E94FD
:10066800A20AE0E00E94A90AA1D1E0917408E7700B
:10067800E09373087894EFEFE0937A0812DFFECFE7
:10068800FFCFA0E8B8E00E94AE0A08951A930A9333
:10069800F89400918008109181087894F8010991E4
:1006A800199108951A930A93F1DF8F01EA81FB816A
:1006B800AC81BD81EA0FFB1FE01BF10BDF010E943B
:1006C800020C14F4E0E001C0E1E0198108812696EB
:1006D8000895A881B981AF30E7E2BE0721F40E94EE
:1006E800B40AA3E003C00E94B40AA1E0A083AC81CD
:1006F800AA2372F00E94BC0AEA5FFA4FAB81BC8160
:10070800A083B1830E94BC0AEB5FFA4FA0E010C03F
:100718000E94BC0AEA5FFA4FDF01EB81FC810E946C
:10072800930BED93FC930E94BC0AEB5FFA4FA1E098
:10073800A0830E94BC0AEC5FFA4FAA81A0830E94A2
:10074800BC0AEE5FFA4FA881B981A083B183E0911A
:100758004805EA9304D0E09348050C944108E881E1
:10076800EF5FE883A881A83010F0E0E0E883E88133
:100778000C94CF08A0914905BB27E0914805F0E00B
:10078800319606C0A0914805BB27E0914905F0E0E5
:100798000E94FB0BEA1BFB0B3896DF01E8E0F0E058
:1007A8000E94D20B08950E94080C31E00E94C20AF0
:1007B800A03320F00E94C20AA43308F028C030E019
:1007C8000E94C80AE270E6951E2F0E94C80AE170CE
:1007D8000E2FA0916B081A1729F4E1E0EA27E0939D
:1007E8006B0831E0A0916C080A1729F0E1E0EA27CC
:1007F800E0936C0831E0E0916C08EE0FE05DA091A9
:100808006B08EA0FEA930E94F6070E94CE0AE32FCC
:100818000C94F2071A9310E00E94D10AE12F0C946D
:100828007B0726970E94060C0E94AE07E13010F461
:100838000C946E04A0915308AB3421F4E091540851
:10084800E33209F003C00E94C6071E2FA091530887
:10085800A23421F4E0915408E63409F012C00E9451
:10086800D80A21F00E94C607EA87FB87EFE0F7E283
:10087800E417F50719F40E94E50A02C00E94F00A7D
:1008880028DFA0915308A33421F4E0915408E634FA
:1008980009F012C00E94D80A21F00E94C607EA8710
:1008A800FB87EAEFF0E0E417F50719F40E94E50A80
:1008B80002C00E94F00A0DDFA0915308A23421F46F
:1008C800E0915408E13209F003C00E94E50A01DF13
:1008D80020D3AACF0E94D10A0E940D0C2D9608950C
:1008E8001A93E2E5F7E0E0936F08F0937008ECE400
:1008F800F5E0E0937108F09372080E94D10A0E9413
:10090800F80AE43421F00E94F80AE33479F40E94EA
:10091800FE0AAE2FE0917308E05DEA1721F00E940D
:10092800FE0AEA3219F426DFE43008F43DC00E94DA
:10093800040B0E94F80A0E94070B0E94FE0A0E94FC
:10094800070BA0917108B09172081C91E091710891
:10095800F09172083396E0937108F0937208E12FD2
:10096800EF3071F4A0916F08B09170081397EEE022
:10097800EC9319DFE13019F4E0E0EA934BDF0FC0A4
:10098800EE3069F4A0916F08B09170081397EFE00A
:10099800EC9309DFE13019F4EFEFEA9342DF0E94AC
:1009A800D10AE1E00C94B4080C94B308EFEFE0939B
:1009B8006908E0936A080895AC81A03310F0AA335F
:1009C80008F006C00E940D0BE0530E94150B55C39A
:1009D800AC81A13410F0A73408F006C00E940D0BBA
:1009E800E7530E94150B49C3A881B981E0E0EC9355
:1009F80044C30E941F0B1A930A931BB10CB1E091D8
:100A0800B708F0E0EB57F74F0083A091B708AF5F46
:100A1800A093B708A23319F4E0E0E093B70809916E
:100A2800199139C21A93E091B808A091B708EA174A
:100A3800D1F3F0E0EB57F74F1081A091B808AF5F02
:100A4800A093B808A23319F4E0E0E093B808E12FC6
:100A580087C3E091B808A091B708EA1709F08FC2D8
:100A68006DC30E941F0BE0911E09A0911D09EA1792
:100A780051F0A0914C06A03029F0A0E00A99A1E01D
:100A8800A03009F401C00CC00E94250BA0911E09DA
:100A9800AF5FA0931E09A43619F4E0E0E0931E09A5
:100AA800FAC11A93E0911E09A0911D09EA1761F491
:100AB8005D9B0AC0A0914C06A13029F4A0E00A99D8
:100AC800A1E0A13009F013C010911D090E942D0B5F
:100AD800E754F74FA981A0831F5F143609F410E08B
:100AE800E0911E09E117E1F310931D0902C0E981A5
:100AF800ECB9FDC1E0E0E0931E09A0911D09A13009
:100B080038F00E94250BE0911E09EF5FE0931E0963
:100B180008950E94080C9DDFE03011F40C94EB0559
:100B280081DF1E2FA0918408A53618F0E0E0E0933D
:100B38004D06E0915106E03011F00C94EA05E09181
:100B48004D06E030A9F4123069F4E1E0E0934D0677
:100B58001093500610935206E0934E06E6E0E09399
:100B68004F0605C010935206E7E5E09351062EC0E4
:100B7800E130C9F40E94300B1083E12FA091500698
:100B8800EA27E0935006E0914E06EF5FE0934E06A9
:100B9800E0914F06E150E0934F06E03019F4E2E0AF
:100BA800E0934D0613C0E23089F4133021F4A0918C
:100BB8005006A03009F007C0E7E5E09351060E940F
:100BC800300BA0E0A083E0E0E0934D06A4CF06C27E
:100BD800AA93BA93EA93FA93EFB7EA931A930A930C
:100BE80010919B0000919C00E12FEC71A9F4E09119
:100BF800E709F091E809E15EF64F0083A7EEB9E056
:100C08000E94AE0AE83CA0E0FA0731F4E0E0F0E028
:100C1800E093E709F093E80909911991E991EFBF89
:100C2800F991E991B991A99118951A930E94360BF7
:100C38000E943B0BD9F30E94360BE15EF64F108100
:100C4800A9EEB9E00E94AE0AE83CA0E0FA0731F448
:100C5800E0E0F0E0E093E909F093EA09E12F80C2CF
:100C68000E94360B0E943B0B09F089C167C20E94A3
:100C7800080CF6DFE03021F0A0918308A03009F0DD
:100C8800E1C0D3DF1E2FA091F309A53618F0E0E0EC
:100C9800E093ED093091ED09E091ED09E03059F468
:100CA800113019F4E4E0E093ED091A3519F4EAE09B
:100CB800E093ED09BFC0E430C1F4E0E0E093ED0952
:100CC8001A3229F0E0917308E05DE11769F4109396
:100CD8004C051093EE09E5E0E093ED09E0E0E093C0
:100CE8008308E1E0E093F009A5C0E530A9F4E0E06D
:100CF800E093ED09E0917308E05DE11761F00E946F
:100D0800420B0E944B0BE091F009EF5FE093F00972
:100D1800E6E0E093ED098EC0E63091F4E091F00949
:100D28000E944B0B0E94420BEF5FE093F009E0E05A
:100D3800E093F109133019F4E7E0E093ED097AC084
:100D4800E73011F0E83059F41A93E1EFF9E0FA933B
:100D5800EA93EDEEF9E0FA93EA932EDE6BC0E93000
:100D680081F4E0E0E093ED09173131F4E091F10905
:100D7800A091EE09EA1709F003C0E4E5E0938308BF
:100D880059C0EA3041F4103011F4EBE001C0E0E062
:100D9800E093ED094FC0EB3071F4E0E0E093F00927
:100DA8001093EF091093EE09ECE0E093ED09E0E011
:100DB800E09383083FC0EC3081F5E091F0090E9490
:100DC8004B0B0E94420BEF5FE093F009E091EF09B3
:100DD800E150E093EF09A091EF09A03021F4A09130
:100DE800EE09A03009F00CC0EDE0E093ED09E091C8
:100DF800F009E1500E94500BE091F0090E94500B5D
:100E0800A091EF09A03021F4A091EE09A03009F4D7
:100E180003C0E0E0E093ED090DC0ED3059F4E0E0E7
:100E2800E093ED091D3031F4EAE5E0938308EFEF34
:100E3800E0938208E091ED09E31719F0E0E0E09310
:100E4800F30917CFCBC00E941F0BE091F50AA091C0
:100E5800F40AEA17E9F0E0914B05E03019F0E8945C
:100E680021F815C0E091F50AF0E0EC50F64FE0816A
:100E7800E0939C00E091F50AEF5FE093F50AF0E05B
:100E8800E030A1E0FA0719F4E0E0E093F50A03C0C6
:100E9800E89420F821F8E991EFBFF991E991A99137
:100EA80018951A93E091F50AA091F40AEA1721F42B
:100EB800E0919B00E072C1F4E091F40AF0E0EC509C
:100EC800F64FA981A0831091F40A1F5FA12FB0E00B
:100ED800A030E1E0BE0709F410E0E091F50AE1175F
:100EE800E1F31093F40A03C0E981E0939C001881B0
:100EF80022960895EA93EFB7EA93E0E0E093F50AC3
:100F0800E0917308EF5FE0934B05E991EFBFE9913A
:100F180018950E94C20AA03220F00E94C20AAB3380
:100F280009F403C00E94CE0AF4CF0E94C20AAB3370
:100F380011F40E94CE0A08950E94C20AE881EA17B5
:100F480031F40E94CE0A3197E1E00C94CF08E0E03A
:100F58000C94CF080E94C20AA03220F00E94F80A1E
:100F6800E03208F40EC00E94C80AE09353080E94B9
:100F7800CE0A0E94C80AE09354080E94CE0AE1E013
:100F88000895DCC00E94080C00E010E00E94C20A2C
:100F9800AD3229F40E94CE0A2FEF3FEF02C021E0C4
:100FA80030E00E94C20AA03320F00E94C20AAA338D
:100FB80008F010C0D801EAE0F0E00E94A40B0F018D
:100FC8000E94C80AE053F0E0E00DF11D8F010E9475
:100FD800CE0AE7CFF901D8010E94A40B0E940F0C9A
:100FE80024960895E8810E94070BE881A0916D0876
:100FF800EA0FE0936D08E881A0916E08EA27E09374
:101008006E080C94CF081A93E5E5F8E0FA93EA9392
:10101800EAECF0E0FA93EA93EF81F8850E94970BE7
:101028000E94F60B84E00E94280A289610E00E948D
:101038002D0BEB5AF74FE081E03241F40E942D0B63
:10104800EB5AF74FA0E3A0831F5FF1CFA981BA81C4
:10105800EAE0F0E0EA1B1E2F0E942D0BEB5AF74F37
:10106800E081E03049F00E942D0BEB5AF74FE08108
:10107800EA93B8DF1F5FF0CF188125960895E9EB52
:10108800F8E0E0936F08F0937008E2E0EA93AADFD3
:10109800E2E0E0936E0808951A930A93E0916E08CF
:1010A800EA93A0DFE3E0EA939DDFE9EBF8E0A091A3
:1010B8006F08B09170080E94FB0BEA1BE0931D09B2
:1010C80019DD38C01A930A93E0915207E03091F184
:1010D800EAE5EA93E6DEE0E0EA93E3DE10E00E9468
:1010E8002D0BEE5AF84FE081E03011F01F5FF7CF7B
:1010F8001F5F012F0A93D5DE10E00E942D0BEE5AD8
:10110800F84FE081E03079F00E942D0BEE5AF84F4D
:10111800E081EA93C6DE0E942D0BEE5AF84FE0817B
:101128000E0F1F5FEACFE02FE195EA93BADEEDE0FC
:10113800EA93B7DE099119910895EBDCE0E0089590
:101148001A9395DDA0918308AA3549F40E94740486
:101158001E2FB8DFE0E0E0938308E12F01C0E0E054
:1011680019910895A991B991EE27FF276D916623EA
:1011780011F03196FBCF0895AA27BB27E991F99181
:101188000590002011F01196FBCFFD0108955D9B9D
:10119800FECFE881ECB9219608951A930A93AC81A1
:1011A800BD810E94EE0B3097C1F0AA81BB810E94DD
:1011B800EE0B8F01309749F00230E0E01E0760F037
:1011C800F80131978F01ED93FC93AC81BD810E94AA
:1011D800AE0A3197AE81A08303C0EE81EA93D7DFD0
:1011E800198108812796089526970E94060C10E019
:1011F800EA89FB893196EA8BFB8B3197E4912E2F94
:10120800E03011F40C94240AE12FE03039F425324F
:1012180011F411E002C00E94560B11C1E130A9F48B
:10122800253219F40E94560B09C112E040E000E093
:101238002D3211F401E003C12B3211F44BE2FFC04F
:10124800203211F440E2FBC002C0E23039F450E031
:1012580013E0203311F40068F2C004C0E33011F049
:101268000C94230A203310F02A3308F009C0A52F64
:10127800EAE0EA9FF0015E2FE22FE0535E0FDFC045
:10128800E22FE33649F40E94610BE889F989A481C9
:10129800AA930E94670BD2C0E33741F40E94610B06
:1012A8000E94710B0E94B6081E2F0AC0E03761F435
:1012B8000E94610B0E94710B0E94C0081E2F0860DB
:1012C80002600F7730E035C0E43611F0E93611F4EA
:1012D800046002C0E53731F4E8EAF0E0EE83FF830A
:1012E80015E00DC0E83511F4086004C0E83711F0C6
:1012F8000C94220AE2EBF0E0EE83FF8314E002FF95
:1013080014C00E94610B0E947B0BAB85AA233AF4A0
:10131800EA85FB850E94930BEA87FB874DE2403004
:1013280011F01F5F01C00B7F04C00E94610B0E9477
:101338007B0B00FD11C0151778F407FF08C002FFEA
:1013480004C00B7F242F115001C020E301C020E20C
:101358000E94560B5150EFCF312F01FF1AC0303089
:10136800B9F003FF08C0EE81FF813196EE83FF8359
:101378003197E49105C0AE81BF81ED91AE83BF8303
:10138800EA930E94670B503009F051503150E7CF73
:101398004BC020E3EE81FF810E94F20BE887F987BA
:1013A800EE81FF813296EE83FF83E885F985AA8571
:1013B800BB85AE17BF0750F02F5FA885B985EA85B2
:1013C800FB85EA1BFB0BEA87FB87EFCF2A3328F064
:1013D80003FF02C0295F01C0295D04FD1AC0213343
:1013E80020F4A885B985119709F409C0531710F09E
:1013F80000FF01C013C020E207FF0BC020E300611B
:1014080002FF07C00B7F4A930E94670B503009F018
:1014180051500E94560B503009F051503150A88558
:10142800B985129708F0B5CF00FF08C0503031F0E9
:101438005150E0E2EA930E94670BF8CF10E0D8CE53
:101448000E940D0C64960895FF92F82E22971A9325
:101458000A93DE010E948F0B8D01DE0116960E9411
:101468008F0B0E94EE0BEA83FB83DE0114960E9429
:101478008F0B0E94EE0BFA93EA931A930A93FE01DC
:101488003696FA93EA93E0E0F0E0FA93EA93ACDE5A
:10149800AA81BB81E0E0EC93198108812496FF9032
:1014A8000895E0934A050E944A03E0937E08F0936A
:1014B8007F080895E0914905A9E0EA9FF0010895A1
:1014C800E050FB4F9F01D9011196EC91E13008954E
:1014D800E0914905EA930E94B303E0934905089512
:1014E800E0917E08F0917F08FA93EA930895FA93C1
:1014F800EA930E945603E03008950E944308E09161
:101508007408E295EF70EC59EA930C94F607F0E052
:10151800FA93EA93E2E0F0E0FA93EA930C9407086E
:10152800EA930E94F6070E945008E1E0BACFE091E2
:101538007B08EF5FE0937B08EFEF0895E091770871
:10154800EA93E0917808EA930895EA93E0E0EA9351
:101558000C94A200ED91FD913196FE93EE930895BF
:10156800E0914805A9E0EA9FF001EF5FFA4F08957E
:10157800E0914805A9E0EA9FF0010895A09171085B
:10158800B0917208AC910895A0917108B091720859
:10159800EC910895A1E7B8E0DDCFA0916F08B09174
:1015A8007008E0E0EC9308950E94C607AF01E1E0FF
:1015B800F0E0EA87FB87EAE3EA930E94A007E030BD
:1015C8000895E1E0F0E0FA93EA93E0E0EA93EFE0CF
:1015D800F7E2FA93EA930895EA85FB85FA93EA938A
:1015E8001A935A934A930895E0917108F0917208FA
:1015F800E1810895E0917108F0917208E2810895FF
:10160800AFE6B8E0A7CFA0916F08B0917008EC934F
:10161800F7CFAA81BB81EC91E295E07FAE2FEC81F8
:101628000895EA0FAA81BB81EC93A881B981EC9156
:10163800EF5FEC930895AA93EA93FA93EFB7EA93CE
:101648000895E0911E09F0E0E754F74FE081ECB906
:101658000895E12FF0E00895E0914E06F0E0EE5A8B
:10166800F94F0895E091E909F091EA090895A091E8
:10167800E709B091E809EA17FB070895E12FA0915F
:10168800EE09EA0FE093EE09E091F0090895F0E021
:10169800E45BFA4F10830895F0E0E45BFA4FA0E0B2
:1016A800A08308952A93EF85F889FA93EA93FE01B7
:1016B8003F96FA93EA930C94D108E889F98934970C
:1016C800E88BF98B0895EF85F889FA93EA93FE0180
:1016D8003F96FA93EA930C94D108A889B98914968D
:1016E8000E94EE0BEE83FF83FA93EA930895A8898C
:1016F800B98914960E94EE0BEA87FB870895E99151
:10170800F991309639F080EA9FE00197F1F7A895B2
:101718003197C9F708950024AF0DB01D0895F195CC
:10172800E195F04008956F2F660F660B762F0895A8
:10173800FA9FF02DEB9FF00DEA9FE02DF10D089533
:101748003BD0F6DF0EF4EBDF0895002498E0AA0FF3
:10175800001C0E1A10F40E0E01C0A1609A95B9F77C
:10176800EA2FA02D08950024112490E1AA0FBB1F91
:10177800001C111C0E1A1F0A18F40E0E1F1E01C0A1
:10178800A1609A9599F7FD01D001089515D0EBDF76
:101798000EF4C5DF0895D9DFEA2F0895E894B7FF5E
:1017A80004C0A095B09511966894F7FDB8DFDBDF0B
:1017B800FD010EF4B4DF0895E894F7FF02C0AFDF2F
:1017C8006894B7FF06C0A095B095119600F80394E9
:1017D80000FA0895ED91FC91119708950590F49100
:1017E800E02D08957A936A93FA93EA9308951B2E4D
:1017F800BF2FF12D1A2EAE2FE12D089500240A16C1
:101808000B0608955A934A933A932A931A930A9384
:1018180008955D814C813B812A8119810881089551
:00000001FF
